:03000000021CC41B
:0C1CC40078FFE4F6D8FD7581E0020036E0
:0100190022C4
:0619F6008B2C8A2D892EC6
:1019FC007572027F48121B61121D09EF20E0F9ABD2
:101A0C002CAA2DA92E120832787BE6FE08E6FDEDF5
:011A1C00FFCA
:011A1D0022A6
:10103B0043525354005341564500434647002D3EFF
:10104B0053320052415445434C5220554E49544261
:10105B004C4E4B5452494754524556535452545389
:10106B00544F505A45524F4241554444464C5453A9
:10107B0041564552535420535720202E3173202E66
:10108B003273202E3573203173202032732020359C
:10109B007320203130732033307320316D20203298
:1010AB006D2020356D202031306D2033306D203197
:1010BB006820200000000100020005000A00140057
:1010CB00320064012C025804B00BB8177046508CD8
:1010DB00A001020408103046656574596172644DB5
:1010EB006574724F6666204F6E20204E6F2020591C
:1010FB006573204F66662054696D65416C7420548E
:10110B007269674F66662054726967507772205216
:03111B00656320E9
:101A440025E024BEF582E43410F58322052EE52E2C
:101A5400C3940222A62EE52E75F004A42208F608EB
:041A6400F608F62268
:10155500789B76AB0876CD08760008760AE408F61F
:1015650008760108F6087664087640121A6108F6CE
:1015750078A9F608760A08F608763C08F60876147F
:1015850008F608760F121A6178B676057BFF7A1091
:0D159500793B1219107F051218720219A07F
:1019420075761D7577C0121679789CE664CD7004A1
:1019520018E664AB600312155578B5E6FFF4600330
:0F196200EF700478B5760178B6E6B4FF0276052B
:011971002253
:0D1C7E00C2AF7DC07C1DE4FF121BECD2AF95
:011C8B002236
:101679007539FF85763A85773B753C00753D007570
:101689003E9BE4FFAB39AA3AA93B8F8275830012CE
:101699000805AB3CAA3DA93E8F8275830012084418
:1016A9000FBF1CE078B4E6FFF46003EF700478B470
:0216B9007601B8
:0116BB00220C
:1019A0007D01E4FF121AEC7BFF7A107940121910C6
:1019B000121C7EC2AF7F9B7B1C7DC07C1D121BF660
:0D19C000D2AF7F02121872E4FDFF021AEC94
:10059200E4F52C7BFF7A1079451219107F051218A9
:1005A20072A297829650FAA2969218A2979219E591
:1005B2002C75F004A4244EF9741035F0FA7BFF1266
:1005C20019107F05121872852C2DE4F52E7BFF7A07
:1005D200107949121910E52CB40A00400302066092
:1005E2009005E9F828287302060702066002062829
:1005F20002063002063402063C02064402064802A3
:1006020006500206587F01EF121A44789DE6FC0854
:10061200E6FD7401936D7003E4936C70028F2E0FEC
:10062200BF0FE40206E6789FE6F52E02070978A0DE
:10063200800278A8E6F52E02072378A7E6F52E02B7
:10064200075178B1800278B2E6F52E02076E78B3D0
:10065200E6F52E0207A378B6E6F52E0207C9E52CC9
:10066200652D60030205B1A218309601B35013A2A2
:1006720096921830960C052CE52CC3940D4003E499
:10068200F52CA219309701B350D4A2979219309742
:10069200CDE52CB40D0050C69006A1F828287302AF
:1006A20006C80206F10206F702071502072F020723
:1006B2004302075C0207790207910207B70207DAD1
:1006C2000207E00207E6052EE52EC3940F400375EC
:1006D2002E01E52E121A44E493FF740193789DCF04
:1006E200F608EFF6121A5A2482F974100207AC12B5
:1006F20014AB020660052EE52EC394034003E4F515
:100702002E789FA62EE52E75F004A424E2F974102B
:100712000207AC121A504003E4F52E78A0A62EE58B
:100722002E75F004A424EEF974100207AC121A50CC
:100732004003E4F52E78A8121A5824EEF9741080BA
:1007420069121A504003E4F52E78A7A62EE52E75FD
:10075200F004A424F6F974108050052EE52EC394FB
:10076200044003E4F52E78B1A62EE52E75F004A41C
:1007720024FEF974108033052EE52EC39403400342
:10078200E4F52E78B2121A5824FEF97410801B0573
:100792002EE52EC394044003E4F52E78B3A62EE58D
:1007A2002E75F004A4240EF9741135F0FA7BFF12B1
:1007B2001910020660052EE52EC394064003E4F5E7
:1007C2002E78B6A62EE52E9010DC9375F018A4FFB5
:1007D200AEF012127002066012155502066012196E
:0A07E200A002066043A208020660B0
:0A1CDC004552415300444F4E4500AD
:101C4F00789DE6F55008E6F55122E567AE66780611
:011C5F002262
:1011E400C216C21778B5E6FFE4FCFDFEFB7A20F9CF
:1011F400F81208668F6D8E6C8D6B8C6AE47B40FAF6
:10120400F9F81208F18E648F65E4F52DF52EC3E527
:101214002E9565E52D9564501CE52C64816016AF10
:101224002EAE2D121972121BD88F2C052EE52E709E
:10123400DD052D80D9E52CB48108E52E152E70022C
:10124400152DE52E65657004E52D6564700CD216C8
:10125400121CA8E4F566F5678007852D66852E6760
:0B126400E4F568F569754F80121C4F1F
:01126F00225C
:10197200C3EF9565EE95645024EF7806C333CE33FA
:10198200CED8F9FD757202EE787BF6CFEDCFEF0877
:0D199200F67F50121B96121D09EF20E0F9A0
:01199F002225
:031B7C00CDEFCDDD
:101B7F00757202EE787BF6ED08F67F50121B961207
:061B8F001D09EF20E0F942
:011B9500222D
:101BD8007572017F50121B61121D09EF20E0F97820
:031BE8007BE6FF9A
:011BEB0022D7
:101BC300121B7CE4FFFE0FBF00010EBE0FF8BFA087
:041BD300F5121BD814
:011BD70022EB
:0618A800CBEFCBCAEECA33
:1018AE00301603301727757203EA787BF6EB08F6CD
:1018BE0008EDF67F50121B96121D09EF20E0F9E499
:0D18CE00FFFE0FBF00010EBE0FF8BFA0F51A
:0118DB0022EA
:1016FF00752F0075300075314FE4F52E121C59C34C
:10170F0033CE33CED8F97C00252EFFEC3EFEAB2F27
:10171F00AA30A931852E82758300120805FD121893
:10172F00A8052EE52EC3940640D27568007569068C
:01173F002287
:101376008E2C8F2D121C59C333CE33CED8F9256946
:10138600FFE5683EFEEEC0E0EFC0E0E52CFDD0E0F4
:10139600FFD0E0FE1218A80569E56970020568121B
:1013A6001C59C333CE33CED8F92569FFE5683EFE16
:1013B600AD2D1218A80569E569700205680553E5A3
:1013C6005370020552C3E5699440E56894004017DE
:1013D600E4F568F5690567E567700205669565E5F4
:0813E6006695644002D2162254
:1014AB00E4F568F5697BFF7A1C79DC121910D21709
:1014BB00E4F539F53AC3E53A9565E539956450217C
:1014CB00E53AAE397806C333CE33CED8F9F5698E0B
:1014DB00687D81FF1218A8053AE53A70D805398066
:1014EB00D4C2177BFF7A1C79E1121910E4F566F56B
:0714FB0067F568F569C216F0
:0115020022C6
:10145200E4F539F53AF53BF53CC3E53C9565E53BEA
:1014620095645044E53A6481603EAF3CAE3B12194C
:1014720072121BD88F3AE53A64807022AF3905396F
:10148200FCFDFEFBFAF9120E127F2C120016AE3B87
:10149200AF3CE4FCFDFBFAF9120E12121CF9053CFA
:0814A200E53C70B5053B80B18B
:0114AA00221F
:0215EE008F3933
:1015F000E4F53AF53BF53CF53DC3E53D9565E53C45
:1016000095645030E53B6481602AAF3DAE3C1219D1
:1016100072121BD88F3BE53BB4800FE53A653970F9
:1016200007AF3DAE3C021972053A053DE53D70C974
:04163000053C80C530
:011634002293
:10174000121C4F78A8E6F554E4F552F5531216FF33
:1017500085666E85676F7F011213EE30021A78ABD3
:10176000E6FE08E6FFE4FCFD7B64FAF9F812086681
:101770008F618E608D5F8C5E300505C205121BADDA
:011780002246
:1018380085662C85672DE56945686008052DE52DC9
:101848007002052C856E66856F671216FF852C66FB
:10185800852D67C3E52D9565E52C95644007E4F56E
:0A18680066F567D2167F020213EE48
:101BEC00740478FF769612FF0322740078FF7696C1
:041BFC0012FF0322AF
:0300330002111E99
:0D111E00C0E0C0F0C083C082C0D075D00812
:10112B00E5D954F8FF120A0A115808115810116723
:10113B0018118220116928118230118438118A40CC
:10114B0011824811A35011C058000011CE8575DAD9
:10115B00C2DDC2DC7573007574008070800EE572A1
:10116B00700280560574E574700205731200268FA9
:10117B00DAC2DDC2DC80558016D2DDC2DC804DC206
:10118B00DDC2DCE5727004C2DA8041D2DA803DC286
:10119B00DDD2DC7570048034AFDA121CD00574E537
:1011AB007470020573C2DDC2DCE5727004C2DA80B2
:1011BB001BD2DA8017AFDA121CD0C2DDD2DC75700D
:0E11CB00028009757004C2DDC2DCD2DAC2DB1C
:0B11D900D0D0D082D083D0F0D0E03224
:1019CD0043910C43920CE4F5DBEF25E0F5DB301889
:1019DD000343DB0175DD2575DC2575D84453F8FE11
:0919ED0053F7FEE4F570D2E82284
:101B9600E57030E002FF22E4F571757003EF25E091
:071BA600F575D2DD7F02227C
:101B6100E57030E002FF22E4F5711572757005EF42
:0B1B710025E04401F575D2DD7F022263
:061D090020DBFDAF70229B
:0D0026001572AF710571747B2FF8E6FF2293
:0C1CD000747B2571F8EFF6057115722287
:0E1C8C00E4F5847585FFF592F5A475A5FF2299
:0E1C9A00EE3395E0FDFC227B007A00791B22E0
:101A6800C213C215C212D2A2C2A0C2A1E4FDFF12C3
:101A78001AECE4FD7F01121AEC7F081213EE7F04C2
:031A88000213EE58
:101AEC00EF146011047016BD0104C2A78002D2A7C6
:0E1AFC00A2A7921422BD0103C2A622D2A622E6
:1013EE00EF14B40800505C90140375F003A4C58389
:1013FE0025F0C5837302141B021421021428021453
:10140E0034021436021434021440021448D21375F6
:10141E00190122C213A21492A722D215751A027DA7
:10142E00017F01021AEC8005C212C28722C212D2BB
:10143E008722D212D28775180122C2A47F011218F8
:04144E0072D2A42290
:1017C000301312D5190F30A707C2A775190F80055E
:1017D000D2A7751923E51AD39400400CD51A09C273
:1017E00015E4FD7F01121AEC301211D5180E308766
:0D17F00006C28775180522D28775181E22C3
:101AAC00C374039FFE1392A0EEA2E192A1AF80CF6C
:0F1ABC005480CFED547FCF4FCF8F80C2A2D2A2E4
:011ACB0022F8
:061910008B3B8A3C893D7F
:10191600E4FCCFECCF7D20121AAC0CBC04F4E4FC42
:10192600AB3BAA3CA93D8C82758300120805FD607D
:0B1936000ACFECCF121AAC0CBC04E589
:011941002283
:041270008F828E8358
:10127400121C9AE47B0F7A27F9F8C31209915003E0
:1012840090270FAF82AE83121C9A7B197AFC79FFE8
:1012940078FFD3120991400390FC19E4F52F741BD5
:1012A400252FF8E4F6052FE52FB405F2AE83AF82BF
:1012B400121C9A121CA1120E12E51E701A752F032D
:1012C400741A252FF8E6FF741B252FF8C6EFC6D530
:1012D4002FEE751B2080E2121CA112191030081584
:1012E4007F811200167F181200167F021200161258
:0512F4001CA1121C3CCE
:0112F90022D2
:101B0A0046554C4C0050524F47005A4C4F47004DD7
:0D1B1A004F440076332D320054726967008D
:101B2700E6FE08E6FFE4FCFD2278D21209CC78CA6B
:0D1B37000209E5C3E55D94B8E55C940B225E
:03001300021A8B43
:101A8B00C0E0C0D075D010200F0CAF8DEFAD8BF533
:101A9B0059EDF55AD20F758D00758B00D0D0D0E073
:011AAB003208
:021872008F3AAB
:10187400E4F53BF53CC3E53C953AE53B9400502345
:10188400900000AF82AE83E4FCFD7B207A4EF9F831
:10189400D31209914003A380EA053CE53C70D605C8
:0318A4003B80D2B4
:0118A700221E
:0E1CA8007BFF7A1B790A1219107F0A0218724C
:0F1C6000D20C301606121CA8C20C2212174022FA
:05000E00C20C021838CD
:101BAD0078D61209F100000000121B3078D212090C
:061BBD00F100000000220F
:10003600121C8C121CE6121A687F04121872209782
:10004600147BFF7A1B790F1219107D017F011212A2
:10005600FAD2AF80FE209612D2AF121942C2187F92
:10006600701219CD1211E41205921219427A1B79F7
:100076001412057D120588D2AF7BFF7A1B791912FF
:10008600191078B4E62430FD7F03121AAC7F0412EF
:1000960018727A1B791D12057DC2187F701219CD50
:1000A6007F011218721211E4120019E4F57A121780
:1000B600FD7F01121872E478DAF608F612001AA229
:1000C600969209A297920AE4F52478CE1209F100D5
:1000D600000000E4F52578D61209F1FFFFD8F17883
:1000E600CA1209F100000000E4F54E78D21209F1B7
:1000F60000000000C20EC20CC20DE4F562F563F505
:1001060026F527C208F55CF55DF559F55AC20FF5D7
:100116005BC210F558F557F556F555F561F560F5DE
:100126005FF55EF52078B1E624FE600B14600C24C2
:1001360002700AD2018006D2068002D20078B2E6A8
:1001460024FE6007047006D2028002D20778B3E666
:1001560024FE600B14600C2402700AD2038006D2BF
:10016600048002D205300117C20178A9121B277B31
:1001760064FAF9F81208668F588E578D568C55E535
:100186007AC3940240F9E4F57AA208B392A6300D38
:1001960033A209309601B3400BA20A309701B3404F
:1001A600030202D830961230970FC20DE4F562F5BD
:1001B600637F041213EEE4F54EA2969209A297927B
:1001C6000A0202D8209605209702D21130965630A0
:1001D6009753301131C21178CA1209CCEC4D4E4FEB
:1001E60078D6700C1209F100000000121B30801046
:1001F6001209F10000000078CA1209F1000000009F
:10020600D20AD209802478A0E6601F0563E56370F0
:10021600020562D394B8E562940B400ED20D7F05B9
:100226001213EE8005E4F562F563A209309601B378
:10023600502DA296920930961F20111C121B3A507F
:1002460017C201E54E6007E4F54E7F068005754E40
:10025600017F071213EE805BE4F55CF55D805420A8
:100266009651740A255DF55DE4355CF55C121B3A22
:100276004041E55D9410E55C94275037755C277521
:100286005D10300807C2081205888027D2087D0154
:10029600E4FF1212FA7F891200167F011218727F8C
:1002A600821200167F011218727F841200167F31A7
:1002B600120016A20A309701B35017A297920A307D
:1002C600971020110DB20C300C05121C6080031221
:1002D600000E120A30AF58AE57AD56AC55EC4D4E27
:1002E6004F602674FF2FF558EE34FFF557ED34FFB7
:1002F600F556EC34FFF555AF58AE57AD56FC4D4E9E
:100306004F7006200C03121C60AF61AE60AD5FAC8F
:100316005EEC4D4E4F602374FF2FF561EE34FFF512
:1003260060ED34FFF55FEC34FFF55EAF61AE60ADB6
:100336005FFC4D4E4F700312000E200F030203E8C0
:10034600C2AFC20FD2AFE4855A2B85592AF529F5DB
:1003560028AF2BAE2AAD29AC287B107A27F9F812E4
:1003660008668F2B8E2A8D298C28E4FB7A90F9F863
:100376001216358F2B8E2A8D298C2878A7E66009D0
:10038600C374B89FFF740B9EFEE55B14601624FED3
:10039600602024037049C3EF94B0EE9404500E75A8
:1003A6005B018009D3EF9414EE94054035755B0329
:1003B6008030C3EF94B0EE94045027755B01300093
:1003C60006200C03121C60300305C203121BAD305D
:1003D6000C02D2107BFF7A1B79221219108003E4DB
:1003E600F55B0525E525C394015003020577E4F581
:1003F60025FB7A0079DC1219F678DDEEF608EFF6C1
:1004060078DCE66402600302057778CE1209D8E844
:10041600C0E0E9C0E0EAC0E0EBC0E078DDE6FE0857
:10042600E6FF789FE6FD1215A2D0E0FBD0E0FAD0F9
:10043600E0F9D0E0F8EB2FFFEA3EFEE93DFDE83CAF
:10044600FC78CE1209E50524E524C3940550030281
:10045600057778CE1209CCE47B05FAF9F812163541
:1004660078CE1209E578CE1209CC78CA1209D8C31B
:10047600EF9BFFEE9AFEED99FDEC98FC78CE120903
:10048600E578D61209CC78CE1209D8D31209914054
:100496000A78CE1209CC78D61209E5E54E600D78B9
:1004A600D8E6FF08E678DFCFF608EFF678D0E6FF65
:1004B60008E678DDCFF608EFF6E54E600308800221
:1004C60078DDE6FE08E6FF1212700527E5277002C2
:1004D6000526C3789E96E52618964045E4F526F54A
:1004E60027300E0F78DDE608FF12001678DEE6FFED
:1004F600120016300C2B7F031213EE20161D78A85F
:10050600E6600C3010097F007E82121376C21078E6
:10051600DDE6FE08E6FF1213768006121CA812001E
:100526000E78CE1209CC78D21209E578CE1209F1EE
:1005360000000000E4F524300405C204121BAD30AF
:10054600061678AD121B2778D21209D8D312099154
:100556004006200C03121C6030071678AF121B27CA
:1005660078D21209D8C31209915006300C03120032
:070576000E1217C0020185FF
:10057D007BFF1219107F041218722278B6E6FDE483
:05058D00FF1212FA222A
:101A1E00444C0021536967005A4C4F47004D4F44C8
:101A2E0000332D320046656220303320323030369E
:061A3E000050524F47006A
:1016BC00AF34AE33AD32AC31EC4D4E4F22EF24FF94
:1016CC00F534EE34FFF533ED34FFF532EC34FFF541
:1016DC003122E475342075334EF532F53122E47540
:1016EC003401F533F532F53122752E00752F007566
:0316FC00309B22FE
:0F1C6F007F041213EEE4F54EC20DF562F5632209
:100A3000121CB6EF7003020C46121B44EF120A0A96
:100A40000C1F240C2B2A0C31500B77520A68610AB8
:100A5000F9630B4C6C0B52720B4F730B7B740BEFE7
:100A6000760BE97800000C46121C6F7BFF7A1A792E
:100A70001E1219101216DE121CB6EF700A1216BCE6
:100A800060051216C980F01216BC7003020C4612E3
:100A90001B448F2D1215EEE4F5341216EEE47F069A
:100AA000FEFDFCAB34AA33A932A831C31209A7500A
:100AB0001F121BD88F2D120016E5342401F534E4E3
:100AC0003533F533E43532F532E43531F53180CD67
:100AD000121BD88F2DE52D64806016E52D64816092
:100AE00010120016121BD88F2D120016752C0180C3
:100AF00003E4F52CE52C70D8221216F51216EAF54F
:100B00002D1216BC60241216DE121CB6EF700A12EB
:100B100016BC60051216C980F01216BC6003120CD8
:100B200047052DE52DC3941C40D71216BC601A78DA
:100B30009BB6AB0708B6CD03020C287BFF7A1A7967
:100B4000211219107F0A021872020BE6B20E22025D
:100B500014521216F5E4F52DAB2E0530E530AA2F10
:100B60007002052F14F91207ECFF120016052DE58F
:100B70002DC3941C40E22243A20822121C6F752E42
:100B800000752F007530781216EAF52D1216BC602C
:100B9000241216DE121CB6EF700A1216BC60051283
:100BA00016C980F01216BC6003120C47052DE52D06
:100BB000C3940240D71216BC602CAE78AF79EE33E6
:100BC00095E0FDFC78D21209D8C3EF9BF538EE9A78
:100BD000F537ED99F536EC98F535AF3878A5E5376A
:100BE000F608EFF68042021679121C6F0214AB7AF7
:100BF0001A7926120C5B7A1A792B121C3C78B4E60F
:100C00002430FF120016121CF97F761200167A1A91
:100C1000792F120C5B7A1A7933121C3C021CF912E0
:100C20001C6FE478A5F608F60219A0121C6F0215D5
:100C300055121C6F7BFF7A1A793F1219107D017FC4
:060C4000011212FA80FE11
:100C460022121B44AB2EAA2FA930852D8275830054
:100C5600EF120844227BFF121C3C121CF97BFF2278
:0A1CE600E4F5955396BF53A27F2248
:1017FD005389F0438901538FFE758C70E4F58A533C
:10180D00B8FD53B7FDD2A9D28C53890F438990539C
:10181D008FEFF58DF58B4391105392EF53B8F7532E
:0B182D00B7F7D2ABD28ED28AD2AA222B
:03000B00021CF0E4
:091CF000057A758C70758A0032CA
:03001B00021D02C1
:071D0200758D00758B0032A6
:101C00000D0A0030313233343536373839414243EA
:041C10004445460001
:101C1400AF4DAB41AA42A943054D22AF40AE3FAD03
:041C24003EAC3D2273
:1012FA005387BF75985053877FE4F5BABF010543FA
:10130A00A240800353A2BFE4F5BDED14601514603A
:10131A001A14601F1460242404702575BEF075BF6A
:10132A000B802375BEF075BF05801B75BEF075BFB7
:10133A0002801375BE7075BF01800B75BEB0800345
:10134A0075BE30E4F5BF75BD035391FE4392014368
:10135A0091025392FDC21A53B8EF53B7EF43B81034
:0C136A00E478C8F618F678C9F6D2AC2278
:030023000218DCE4
:1018DC00C0E0C0D075D01030981E78C8E6C3940F05
:1018EC00501418E60624B7F8A69978C80618E6C36B
:1018FC00941040027600C298309904C299C21AD052
:04190C00D0D0E03225
:08000300201AFDD21A8F992288
:101ACC0078C8E6D39400401508E60624B7F8E6FF7C
:0F1ADC0078C81608E6C394104005E4F6227F0090
:011AEB0022D8
:03001600020003E2
:101B44007F207E4E78C8E67010D3EF9400EE9400A8
:0C1B54004007EF1F70EE1E80EB121ACC51
:011B60002262
:101C3C001207ECFF600C120016740129F9E43AFA51
:031C4C0080EE2205
:0E1CB60078C8E6D3940040037F01227F00220D
:091CF9007BFF7A1C7900021C3CFF
:0E0E12008F408E3F8D3E8C3D8B418A4289433E
:100E2000E4F54DEC4D4E4F7017E94A4B70057F309D
:100E3000020016121C148F827583007430020F3565
:100E4000121C21EC33502AE5434542454170077F8F
:100E50002D120016800D121C148F82758300742DC4
:100E6000120844121C1F1209838F408E3F8D3E8C46
:100E70003D754C017547007546CA75459A75443BEA
:100E8000E4FFFEFDFCAB47AA46A945A844D31209DE
:100E9000A75003020F20121C1FA8441208F18F4B09
:100EA0008E4A8D498C48EC4D4E4F7004E54C7023B2
:100EB000E54B2430FFE543454245417005120016DD
:100EC000800EAE4D121C168E82758300EF12084400
:100ED000E4F54CAF47AE46AD45AC44AB4BAA4AA98E
:100EE00049A848120866C8ECC8C9EDC9CAEECAC309
:100EF000E5409FF540E53F9AF53FE53E99F53EE533
:100F00003D98F53DAF47AE46AD45AC44E47B0AFAAB
:100F1000F9F81208F18F478E468D458C44020E80F9
:100F2000E542454345416010AB41AA42A943854D86
:080F300082758300E4120844FD
:010F38002296
:100C66000134C35001DBBF68028BBB800344B798D5
:100C76000407B3B004D5AFC805A9ABE00689A7F849
:100C86000775A410086DA02809719C400A81985820
:100C96000B9F94700CCA90880DE98CF90E048CA0F9
:100CA6000EA88AAC0F4D88B80FF786C410A184D061
:100CB600115182DC120580E812BB7EF413747D00AC
:100CC60014307B0C14F2791815B877241680753019
:100CD600174B733C1819714818ED6F5419C46D60A1
:100CE6001AA16B6C1B7E69781C6167841D4A65902E
:100CF6001E37639C1F2561A8201A5FB421125DC0B0
:100D0600220D5BCC230E59D8241557E4251F55F028
:100D1600262F53FC27425208285B501429764E2072
:100D26002A9B4C2C2BC04A382CEE48442E1E46508B
:100D36002F55445C308F426831D1407433173E8062
:100D460034633C8C35B13A98370938A4386636B0E6
:100D560039C734BC3B2D32C83C9D30D43E0F2EE003
:100D66003F882CEC41062AF8428D290444182710A6
:100D760045AB251C4741232848E121344A861F40BC
:100D86004C311D4C4DE21B584F9C1964515D177038
:100D96005323157C54EF138856C4119458A20FA000
:100DA6005A830DAC5C6D0BB85E6009C4605807D001
:100DB600625A05DC646203E8667301F4688A00001F
:100DC6006AA1FE0C6CB8FC186ECFFA2470E6F830F7
:100DD600000000000000000000000000000000000D
:100DE60000000000000000000000000000000000FD
:100DF60000000000000000000000000000000000ED
:0C0E0600000000000000000000000000E0
:1017810075F004E533A42466F582E5F0340CF583A5
:10179100E49322FE740193FF75F004E533A422F56E
:1017A10083C37401939FFFE4939EFEE4228F348EE2
:0F17B100338D328C31228F308E2F8D2E8C2D2246
:101C2800C3EF9DEE9C400AD3EF9BEE9A50037F01D1
:041C3800227F0022E5
:040F39008E318F3234
:100F3D00E4F533121781FC740193FD121799246A9D
:100F4D00F582E5F0340CF583E493FA740193FBAF6D
:100F5D0032AE31121C28EF700302102912178112C4
:100F6D001794246AF582E5F0340C1217A08F378E92
:100F7D0036F535F534121799246CF582E5F0340CFD
:100F8D00F583E4931217942468F582E5F0340C127E
:100F9D0017A08F3B8E3AF539F538AD39AC381209BB
:100FAD00838F3B8E3A8D398C38AE31AF32E4FCFDF8
:100FBD00EEC0E0EFC0E0121781FE740193FBCAEEA4
:100FCD00CAD0E0FFD0E0FEC3EF9BFFEE9AFEED949A
:100FDD0000FDEC9400FCAB3BAA3AA939A8381208E5
:100FED0066AB37AA36A935A834121635C8ECC8C970
:100FFD00EDC9CAEECACBEFCB1217992468F582E57D
:10100D00F0340CF583E493FE740193FFE4FCFDEBE7
:10101D002FFFEA3EFEED39FDEC38FC220533E533BA
:0D102D00C3946A5003020F40E4FFFEFDFC77
:01103A002293
:01001A0022C3
:101503001217AEAB34AA33A932A831E8C0E078A3EE
:10151300E6FE08E6FFE4FCFDD0E0F81208661217C9
:10152300AE780E1209B81217AE78A5E6FE08E6FFEC
:10153300EE3395E0FDFCE5342FF534E5333EF5332A
:10154300E5323DF532E5313CF531AF34AE33AD3202
:02155300FC2278
:0215A2008D2C8E
:1015A400120F391217B71215031217B7E52C14606E
:1015B4001C14702DE47FE87E03FDFCAB30AA2FA938
:1015C4002EA82D120866E47BE87A0B800CAF30AEAF
:1015D4002FAD2EAC2DE47B03FAF9F8121635121751
:0915E400B7AF30AE2FAD2EAC2DD7
:0115ED0022DB
:1007EC00BB010689828A83E0225002E722BBFE020B
:0907FC00E32289828A83E493223E
:10080500BB010CE58229F582E5833AF583E02250A8
:1008150006E92582F8E622BBFE06E92582F8E222F2
:0D082500E58229F582E5833AF583E493220C
:10083200BB010689828A83F0225002F722BBFE01A5
:02084200F3229F
:10084400F8BB010DE58229F582E5833AF583E8F0EA
:10085400225006E92582C8F622BBFE05E92582C896
:02086400F2227E
:10086600E88FF0A4CC8BF0A42CFCE98EF0A42CFC31
:100876008AF0EDA42CFCEA8EF0A4CDA8F08BF0A4AF
:100886002DCC3825F0FDE98FF0A42CCD35F0FCEB0E
:100896008EF0A4FEA9F0EB8FF0A4CFC5F02ECD39D3
:0F08A600FEE43CFCEAA42DCE35F0FDE43CFC2240
:1008B50075F008758200EF2FFFEE33FECD33CDCCFA
:1008C50033CCC58233C5829BED9AEC99E58298407D
:1008D5000CF582EE9BFEED9AFDEC99FC0FD5F0D65A
:1008E500E4CEFBE4CDFAE4CCF9A88222B800C1B984
:1008F5000059BA002DEC8BF084CFCECDFCE5F0CBC2
:10090500F97818EF2FFFEE33FEED33FDEC33FCEBFA
:1009150033FB10D703994004EB99FB0FD8E5E4F9B5
:10092500FA227818EF2FFFEE33FEED33FDEC33FCA2
:10093500C933C910D7059BE99A4007EC9BFCE99A96
:10094500F90FD8E0E4C9FAE4CCFB2275F010EF2FDB
:10095500FFEE33FEED33FDCC33CCC833C810D707DB
:100965009BEC9AE899400AED9BFDEC9AFCE899F816
:0E0975000FD5F0DAE4CDFBE4CCFAE4C8F922A9
:10163500C2D5E830E70FB2D5E4C39BFBE49AFAE4E0
:1016450099F9E498F8EC30E717B2D512166B120841
:10165500F1E4C39BFBE49AFAE499F9E498F8800372
:101665001208F130D50DE4C39FFFE49EFEE49DFD15
:04167500E49CFC22D3
:0E098300C3E49FFFE49EFEE49DFDE49CFC2285
:10099100EB9FF5F0EA9E42F0E99D42F0EC6480C8DD
:0609A10064809845F0227D
:1009A700EB9FF5F0EA9E42F0E99D42F0E89C45F0A6
:0109B700221D
:1009B800E86010ECA2E713FCED13FDEE13FEEF1355
:0409C800FFD8F02242
:0C09CC00E6FC08E6FD08E6FE08E6FF2257
:0D09D800E6FB08E6F908E6FA08E6CBF8228F
:0C09E500ECF608EDF608EEF608EFF6223E
:1009F100D083D082E493F608740193F608740293CD
:090A0100F608740393F674047303
:100A0A00D083D082F8E4937012740193700DA3A37B
:100A1A0093F8740193F5828883E47374029368608F
:060A2A00EFA3A3A380DF8F
:00000001FF
